:10000000EEC0189501C01895AFB6B12EC22E1FEFE5
:1000100018BB132F1770103021F4242F919A919848
:100020000EC0113009F4252F123009F4262F133099
:1000300009F4272F143009F4282F909A9098203033
:1000400011F427ED25C0213011F422E121C0223026
:1000500011F42BEC1DC0233011F42BE519C0243012
:1000600011F42EE115C0253011F42DE511C0263014
:1000700011F42DED0DC0273011F423E109C0283013
:1000800011F42FED05C0293011F42FE501C020E057
:10009000033028F4003019F0133009F420621430D2
:1000A00011F436FD2062209528BB13951530D8F049
:1000B00010E03062F030B9F0F395FA3FA0F0F0E0D4
:1000C000202F220F220F220FE3FB22F9E4FB21F95C
:1000D0002EBB0DBAE19AE199FECF23952EBB1DBA36
:1000E000E19AE199FECF387F312B33FF41C0377F52
:1000F000802D712D033040F4003031F076958795D6
:10010000769587957695879544275527662780317C
:1001100017E2710720F0439580517742F8CF883E6F
:1001200013E0710720F05395885E7340F8CF843652
:1001300010E0710720F0639584567040F8CF8A3044
:1001400018F073958A50FBCF033008F011C0152FBB
:10015000412F162F512F172F612F182F712F102D70
:100160001770143008F01395812F003009F48BE0DC
:100170001B2D2C2DAFBE1895282D192D033008F4FA
:1001800010C0043059F0053061F026191709220F0C
:10019000111F220F111F220F111F03C0220F111F49
:1001A00000C0BD2DBF3B11F0220F111F0895E0309C
:1001B00009F008950214130408F002C0042C152C51
:1001C0004014510408F00895022C132C08951EBB0E
:1001D000E09A2DB313950895909A90980895B7D00A
:1001E00033279927002710E017BB1FEF18BB13E038
:1001F00011BB1CE712BB919A9198EEDFEDDFECDFAB
:10020000EBDFEADFAFEFA4D0E6B3E095919A9198E7
:100210001FEF17BBE0FB02F9E1FB01F9E2FB00F97C
:10022000003009F4E0E0E87110E0D1DFD22E102FA9
:10023000110F110F110FCBDF822EC9DF922EC7DFF6
:10024000222EC5DF322EC3DF422EC1DF522EBFDF8A
:10025000622EBDDF722EE03019F4082C192C0CC070
:10026000E83019F4042C152C07C0E03119F4022CE5
:10027000132C02C0062C172C386013E013BF12E0B9
:1002800019BF789444D010B31C711C3189F190309F
:1002900079F035FF2EC03F7D9395983738F4903232
:1002A00040F1292F287F291719F023C097EC00C0AF
:1002B000903031F491E012FD03C020E4322727C0D2
:1002C0000030C1F012FF15C021E0033008F422E035
:1002D00013FD07C014FD00C0020E08F4139467DF7D
:1002E00004C0021A08F41A9462DF3860F1E00FC00B
:1002F0009927C9CF202D2F3B29F02FEB022E23E188
:10030000122EF3CF27E8022E25E1122EEECFE03099
:1003100019F4802C912C0CC0E83019F4402C512C8D
:1003200007C0E03119F4202C312C02C0602C712C54
:1003300023DFC2EC14D0B12F16D0B22F14D0BEE8F8
:1003400012D0B0E036FDB0EE0ED04ED09CCFA4E17E
:10035000AA95F1F70895AAE0AA95F1F70895BC2FA0
:100360008E9A9698F8DF0894BB1F01C0BB0F79F0F6
:100370008D9A959820F40000969A8E9803C08E9AD4
:10038000969800C0E4DF959A8D98E1DFEFCF8D9AC3
:100390009598969A8E98DBDF959A8D98859BFECFDF
:1003A000889486990894D3DF0895C0FFDCCFDD1FC1
:1003B000B1E08D9A9598CBDF959A8D98C8DF889497
:1003C00086990894BB1FA8F78D9A9598D79518F42D
:1003D000969A8E9802C08E9A9698B9DF959A8D98C3
:1003E000859BFECFB4DF08958D9A95988E9A969846
:1003F000AEDF959A8D98AFDF969A8E98A8DF089514
:10040000BF13000000000000884A8048904C0000A4
:10041000B027C026A02800000A28102704298C2312
:100420000A281027042900000A28102704290000A0
:1004300000000000000000000000000000000000BC
:00000001FF
